:03000000020040BB
:03000B0002035895
:030013000203469F
:03002300020330A5
:10004000758130C200C201C202D203C204C205C21D
:100050000775A0017400D2D3D2D47F007E007D004A
:100060007C007B007A0075A890D2BC759850E5871B
:10007000D2E7F587758DE6758920D28EE51DB4002F
:1000800000D2D4D2D3BD2905E51C02008FE51DB4F2
:10009000314A200123D2060200E5D201D2AAD2BA07
:1000A000D2A7C206200532900CA01202911202B70C
:1000B00030042612026D8021C201C202C206C207AC
:1000C000C2AAC2BAD2A0C2A7C2A620050C900CC078
:1000D00012029130040312026D12028030070302F3
:1000E0000231B4326920023130B51BD202D2A620CF
:1000F0000659200551900CE01202911202B730040B
:100100004512026D8040C206900DC012029112028B
:10011000B730043212026D802D20062F200118C244
:1001200002C2A6200520900D001202911202B730E3
:10013000041412026D800F900DE01202911202B7AA
:1001400030040312026D120280800302015730074F
:1001500003020231B4335220031C0202BED2032038
:10016000064420053C900D201202911202B7300483
:100170003012026D802B20062D2001160202EBC2E8
:100180000320051D900D4012029130041412026DDF
:10019000800F900DE01202911202B7300403120298
:1001A0006D120280800302009A300703020231B40C
:1001B0003431200418D204D2A412026D20052190FB
:1001C0000D601202911202B712026D8013C204C2B6
:1001D000A4751600200509900D801202911202B735
:1001E000120280300703020231B4350312043A30A0
:1001F0000703020231B43609200504D2058002C289
:1002000005300703020231B43709900F2012029122
:100210001202B7300703020231B43838900F40128F
:1002200002911202B7900F601202911202B73007CA
:1002300023C2AAC2BA75A0F175892112025975A00C
:1002400000120259D2D4D2D3BD290302007CBC587B
:10025000E002007CD21502007CC28CC28D758C003D
:10026000758A00D28C308DFDC28CC28D22C0E09088
:1002700080007401F0D0E0D28C900C4012029122E8
:10028000D2D4D2D37F007E007D007C007B007A0038
:1002900022C0E0740093B4240A201318740D1202D3
:1002A000A980111202A9A380EAF599D2003099FD24
:1002B000C299C200D0E022BD4BFD12028022758996
:1002C00021D2D4C2D37C00900C00D2D4C2D37D0002
:1002D000C0E0ED93F59012031CD2D4C2D30DEDBD56
:1002E00004F10CBC0AE1D0E002015D758921D2D491
:1002F000C2D37C00900C20D2D4C2D37D00C0E0EDEC
:1003000093F59012031CD2D4C2D30DEDBD04F1D2EB
:10031000D4C2D30CBC0ADDD0E002017FC28CC28DF6
:10032000758C3C758AAFD28C308DFDC28CC28D220B
:10033000200012D2D3D2D4AA1BAB1CAC1DAD1EAE72
:100340001FAF99C2983230B3FD30010B900DA0124F
:100350000291C20475160032C28CC28DC0E0E0F575
:1003600016D0E032E516D2D4C2D37F027519CD750E
:10037000F03384F550C5F0B4000875510075520093
:100380008038BF0002803375F005A475F03384F522
:100390001A7402A48000F51B251930E70DE51A75C3
:1003A000F002A4F5511FE51B800EF51BE51A75F050
:1003B00002A404F5521FE51B80C8E550540F4430D9
:1003C000B4300C74321202A974321202A98049B4FA
:1003D000310C74321202A974331202A9803AB43279
:1003E0000C74321202A974341202A9802BB4330C9B
:1003F00074321202A974351202A9801CB4340C7430
:10040000321202A974361202A9800DB4350A743270
:100410001202A974371202A9742C1202A9E55154D0
:100420000F44301202A9E552540F44301202A9744D
:10043000F81202A974431202A922C0E0900FD01250
:100440000291D213901000120291C2133001089051
:1004500010201202918006901040120291D2139047
:100460001060120291C213300208901080120291A3
:1004700080069010A0120291D2139010C012029127
:10048000C21330030890110012029180069010E010
:10049000120291D2139011C0120291C213200508CA
:1004A00090118012029180069011A0120291D21335
:1004B000901120120291C21330041DD213901140EA
:1004C000120291C21374281202A9120364D2147486
:1004D000291202A9742E8006901160120291740DE7
:0E04E0001202A9741A1202A9D0E01202B72269
:040C000003090C06D2
:040C2000060C0903B2
:0C0CA00041542B434D53533D3239342452
:0C0CC00041542B434D53533D3239352431
:0C0CE00041542B434D53533D3239362410
:0C0D000041542B434D53533D32393724EE
:0C0D200041542B434D53533D32393824CD
:0C0D400041542B434D53533D32393924AC
:0C0D600041542B434D53533D333030249D
:0C0D800041542B434D53533D333031247C
:100DA00041542B434D53533D3330322420242024CF
:0C0DC00041542B434D53533D333033243A
:0C0DE00041542B434D53533D3330342419
:0C0C400041542B434D53533D33303524B9
:0C0F200041542B434D53533D33303624D5
:0C0F400041542B434D53533D33303724B4
:0C0F600041542B434D53533D3330382493
:100FD00041542B434D47533D226E756D2E20646F57
:100FE0002063656C2E64657374696E6F222C3132D8
:030FF0003924247D
:09100000416C61726D653A202417
:0D102000486162696C697461646F2E202460
:0F1040004465736162696C697461646F2E20246A
:09106000506F727461733A202490
:0B10800054726176616461732E2024BD
:0E10A00044657374726176616461732E20245E
:0910C000566964726F733A202432
:0A10E00041626572746F732E2024C4
:0B1100004665636861646F732E202455
:0C112000417175656365646F723A2024AC
:081140004C696761646F202413
:0C1160004465736C696761646F2E202485
:1011C000534D5320646520636F6E6669726D616371
:0511D000616F3A2024CC
:051180004F4E2E20245B
:0611A0004F46462E2024FC
:00000001FF
